:020000040000FA
:100400009D2C08000800080009003D001018422B30
:10041000901D08000F088700901120007839031DF7
:1004200000340719CA322008343A031D1032A001E3
:10043000A401B901B813C01BB8175022090F0F321D
:100440003D000E1220000C3049220C3003322009EE
:1004500040390838A0001030A100A0170800090397
:100460002000B900C708031D0532460203180232F6
:100470004608B9000408BA000508BB003D000E128A
:100480002000C01F0932E92248302A2224094039BD
:100490000838A400A4170800A413A5010C30F533F4
:1004A000833085008E308400400803196A2A013A9F
:1004B00003197A2A203A03197F2AA13A0319852AB7
:1004C000013A0319922A203A0319A42A613A03191E
:1004D000A82AFF34410B0034FE3E03190034FE3ECF
:1004E00003190034FC3E031DFF344208B8000830F5
:1004F000AC0000344108F53E031DFF3400344108D0
:10050000F73E031DFF344208D32C4108031902347F
:10051000063A03192B320E3A031DFF340131381805
:10052000013101344108031902340A3A0319013434
:100530000C3A031DFF344308223A031DFF34833075
:100540008500683084002B34410BFF344208EB2CCB
:10055000410B0532843085002E3084002432090B93
:10056000FF3483308500D2308400B234430B05322F
:10057000833085007F3084001632090B05328330CA
:100580008500883084003234090B0F3284308500B6
:100590005B308400C20A053200080936840703185C
:1005A000850AC20BF93300080800F43E031DFF342E
:1005B00083308500A53084003934B81F0232E92227
:1005C00065334108053A031D080042083D009600C6
:1005D0000800A501B908031908003A0884003B087F
:1005E00085004030860087018310B8188314251ACF
:1005F0001D32851F1632230083180F32950104081F
:100600009100050892001514000000001408343A07
:10061000031D8314130801310232831014082000D3
:10062000013212001E00A50AB90BE133B81083187D
:10063000B8140408BA000508BB0008003D000E12FB
:10064000200027223D001018312B901D222B9011E5
:100650002000A01B222B2008343A03190232031079
:100660000800031408002100FC3099001A095139D0
:10067000031DFC33270090309B0042233D008E0178
:100680008E1508003D009001143091008501203046
:100690008400C3243D000E1796010E120E13901D08
:1006A000033290114123FB33163098001A30990021
:1006B0001A309A0020002030A200A6003030AE0090
:1006C0003030B6002030A300A700AF00B700252AC5
:1006D000063FFF340901A1017508950F1500263466
:1006E000FF0085010901810285020902B10285032B
:1006F0000903B102850409049509B102C03412014D
:10070000100200000010C016D927000301020301E7
:10071000090232000201003480320904003400343E
:1007200001340300000409211001000122342B00D0
:10073000070581031000FA34090401000134FF00A9
:100740000005070582031000FA34050F3900023452
:10075000181005003834B63408343434A934093458
:10076000A03447348B34FD34A034763488341534C7
:10077000B6346534000101011C100500DF3460341B
:10078000DD34D83489344534C7344C349C34D234C5
:1007900065349D349E3464348A349F3400000306EB
:1007A000B20002000A00000000000306B2000800C8
:1007B00001000000A800080002000100A0001400D1
:1007C0000300573449344E34553453344234000016
:1007D00000000000000000008400040007002A0060
:1007E00044006500760069006300650049006E0002
:1007F00074006500720066006100630065004700D8
:100800005500490044007300000050007B0039008F
:1008100037003500460034003400440039002D0014
:1008200030004400300038002D0034003300460012
:1008300044002D0038004200330045002D003100F7
:1008400032003700430041003800410046004600B6
:100850004600390044007D00000000002E030134F2
:100860007734773477342E34743475342D346334DC
:10087000683465346D346E34693474347A342E34AB
:10088000643465342F347E346834653468346134BC
:100890002F346534773461342F344F346634653403
:1008A0006E342F34723461347534633468342E34CA
:1008B000683474346D340403070422035400550073
:1008C00020004300680065006D006E006900740040
:1008D0007A002C0020004500570041001803520008
:1008E00061007500630068006D0065006C006400C5
:1008F0006500720030036800650068006100400018
:10090000680072007A002E00740075002D006300EC
:10091000680065006D006E00690074007A002E00AA
:100920006400650008034800490044000E035700B6
:1009300065006200550053004200332321002B3034
:100940008C0037308E0020003B309B004C309C00E8
:100950002C0094011E309500C030960000308500B8
:10096000A03084005030C32421000130C000023088
:10097000D0000330E0000522FE33F00012001E001C
:10098000F00BFC330034F00003011A00F00BFD33D0
:100990000800F000A0308400700803190332083109
:1009A000F00BFD330834023A03191132013A031DEA
:1009B000FF341E230318FF344108FC390319FF34A8
:1009C000E130860041081E00C924BD2400341E23E6
:1009D0000318FF340034090B0832220010308C0653
:1009E00000308500C03084001034090B053200301F
:1009F0008500D03084001034090BFF3400308500AE
:060A0000E03084000A341E
:00000001FF
